:0200000480007A
:100000006F00C004732F2034930F8000630AFF0336
:10001000930F90006306FF03930FB0006302FF038A
:10002000170F0080130F0FFE63040F0067000F000F
:10003000732F203463540F006F004000136E9E53E3
:10004000171F00002320CFFD6FF09FFF732540F1A5
:100050006310050073251030635805000F00F00F82
:10006000130E100073000000130E00009702000032
:10007000938282F973905230735020307350303035
:1000800073504030970200809382C2F7638C020065
:10009000739052109302B01A739022307323203061
:1000A000E39E62F873500030970200009382420191
:1000B00073901234732540F17300203093000000D8
:1000C00013010000B3A12000930E0000130E2000C6
:1000D000639AD14B9300100013011000B3A12000CC
:1000E000930E0000130E3000639ED1499300300040
:1000F00013017000B3A12000930E1000130E4000F6
:100100006392D1499300700013013000B3A1200025
:10011000930E0000130E50006396D1479300000029
:100120003781FFFFB3A12000930E0000130E600083
:10013000639AD145B700008013010000B3A12000ED
:10014000930E1000130E7000639ED143B700008021
:100150003781FFFFB3A12000930E1000130E800023
:100160006392D14393000000378100001301F1FF37
:10017000B3A12000930E1000130E90006394D141A0
:10018000B70000809380F0FF13010000B3A12000AE
:10019000930E0000130EA0006396D13FB7000080BD
:1001A0009380F0FF378100001301F1FFB3A120001D
:1001B000930E0000130EB0006396D13DB70000808F
:1001C000378100001301F1FFB3A12000930E10004E
:1001D000130EC0006398D13BB70000809380F0FFFE
:1001E0003781FFFFB3A12000930E0000130ED00053
:1001F000639AD139930000001301F0FFB3A12000EE
:10020000930E0000130EE000639ED1379300F0FFC1
:1002100013011000B3A12000930E1000130EF00084
:100220006392D1379300F0FF1301F0FFB3A12000D8
:10023000930E0000130E00016396D1359300E00089
:100240001301D000B3A02000930E0000130E100184
:10025000639AD0339300B0001301D00033A1200083
:10026000930E1000130E2001631ED1319300D000B5
:10027000B3A01000930E0000130E30016394D03130
:10028000130200009300B0001301D000B3A12000BE
:10029000138301001302120093022000E31452FEA4
:1002A000930E1000130E4001631ED32D13020000A5
:1002B0009300E0001301D000B3A120001300000060
:1002C000138301001302120093022000E31252FE76
:1002D000930E0000130E50016316D32B130200007F
:1002E0009300C0001301D000B3A120001300000050
:1002F0001300000013830100130212009302200078
:10030000E31052FE930E1000130E6001631CD327FE
:10031000130200009300E0001301D000B3A12000FD
:100320001302120093022000E31652FE930E000007
:10033000130E70016398D125130200009300B000E2
:100340001301D00013000000B3A12000130212001B
:1003500093022000E31452FE930E1000130E80014E
:100360006392D123130200009300F0001301D00028
:100370001300000013000000B3A1200013021200BC
:1003800093022000E31252FE930E0000130E900120
:10039000639AD11F130200009300A0001300000015
:1003A0001301D000B3A12000130212009302200019
:1003B000E31452FE930E1000130EA0016394D11D9E
:1003C0001302000093000001130000001301D0008D
:1003D00013000000B3A120001302120093022000BA
:1003E000E31252FE930E0000130EB001639CD1196C
:1003F000130200009300900013000000130000009F
:100400001301D000B3A120001302120093022000B8
:10041000E31252FE930E1000130EC0016394D11725
:10042000130200001301D00093001001B3A12000BB
:100430001302120093022000E31652FE930E0000F6
:10044000130ED0016390D115130200001301D000E8
:100450009300800013000000B3A1200013021200DB
:1004600093022000E31452FE930E1000130EE001DD
:10047000639AD111130200001301D00093002001F0
:100480001300000013000000B3A1200013021200AB
:1004900093022000E31252FE930E0000130EF001AF
:1004A0006392D10F130200001301D000130000006B
:1004B00093007000B3A120001302120093022000E9
:1004C000E31452FE930E1000130E0002639CD10B36
:1004D000130200001301D00013000000930030014C
:1004E00013000000B3A120001302120093022000A9
:1004F000E31252FE930E0000130E10026394D10912
:10050000130200001301D0001300000013000000CC
:1005100093006000B3A12000130212009302200098
:10052000E31252FE930E1000130E2002639CD105BD
:100530009300F0FF33211000930E0000130E3002E1
:100540006312D1059300F0FF33A10000930E100059
:10055000130E40026318D103B3200000930E000075
:10056000130E50026390D003930000011301E001C9
:1005700033A02000930E0000130E60026314D0011C
:10058000631CC0010F00F00F63000E00131E1E005D
:10059000136E1E00730000000F00F00F130E10000A
:1005A00073000000731000C0000000000000000095
:1005B000000000000000000000000000000000003B
:0405C0000000000037
:1010000000000000000000000000000000000000E0
:1010100000000000000000000000000000000000D0
:1010200000000000000000000000000000000000C0
:1010300000000000000000000000000000000000B0
:081040000000000000000000A8
:040000058000200057
:00000001FF
